:020000040000FA
:04000000CC303A289E
:08000800A000030EA100831209
:1000100005191028831601178312B23081002B288E
:1000200083160113831203140B190310A80DA90DD5
:10003000AA0DAB0DAC0DAC16FF302C02031D2B2806
:10004000FA302B02031D2B2831152A08AF0029088E
:10005000AE002808AD008B100B11210E8300A00EFE
:04006000200E090065
:0C007400203084008001840A80300402E7
:10008000031C3C281230B000902183160C308505EB
:1000900087018312850187010730990000309A009B
:1000A000103083168E008312603083168F00831207
:1000B0000030831691009F008312C83083168100A0
:1000C000831231309000003083168C008312103080
:1000D0008B002F2281018E018F010B118B100B10D1
:1000E0008C018B17812031198420B30B7F280310DA
:1000F00085190314B90DF03039020319092186223C
:10010000722864003210080031110130B7008B13DF
:100110002030370783169B001C141A088312A40092
:100120001030370783169B001C141A088312A30093
:10013000A6000230A6060030370783169B001C1469
:100140001A088312A200A7000130A7068B17321CE1
:10015000AF2822090339A200A309A409A50924088C
:100160002F02031D032923082E02031D0329220841
:100170002D02031D032901303702031DC4283D1839
:10018000C4283D143E14AB2102303702031DCD2894
:10019000BD18CD28BD143E14B72103303702031D0E
:1001A000D6283D19D6283D153E14C3210430370208
:1001B000031DDF28BD19DF28BD153E14CF210530F2
:1001C0003702031DE8283D1AE8283D163E14DB21BE
:1001D00006303702031DF128BD1AF128BD163E1462
:1001E000E62107303702031DFA283D1BFA283D1788
:1001F0003E14F12108303702031D0329BD1B0329DA
:10020000BD173E14FC21B70A093037020318080055
:1002100087280130B600B300B400B500B7008501EF
:100220008701B1138120B30B4129031085190314F1
:10023000B90DF030390203196829B40B4129013096
:100240003702031907220230370203190C22033048
:100250003702031911220430370203191622053020
:10026000370203191B2206303702031920220730F8
:100270003702031925220830370203192A22963043
:10028000B400311D12293111321C4B292D090339BB
:10029000AD00AE09AF092F1C12298E018F010C1C75
:1002A00012290C102E1E12298B1320303707BB0089
:1002B0002F08BA007B2110303707BB002E08BA0088
:1002C0007B2100303707BB002D08BA007B218B173C
:1002D00085018701B70AB60109303702031C1229CC
:1002E0002F2208003E1C08003E101030BB003D08C5
:1002F000BA007B2108008B133A0883161C159A005C
:1003000083123B0883169B0055309D00AA309D0048
:100310009C1464009C1889291C1183128B170800F7
:10032000831610309B001C141A088312BD0083161C
:1003300030309B001C141A088312DE00FF30C80006
:10034000CA15CB15CC15CD15CE15CF15D015D11599
:10035000D215D3150800F130BD05FF30DE05113090
:10036000C405C0000030C200C6005F100800F230B3
:10037000BD05FF30DE050230C405C0000030C200FC
:10038000C6005F100800F430BD05FF30DE05063002
:10039000C405C0000030C200C6005F100800F8307D
:1003A000BD05FF30DE051830C405C0000030C200B6
:1003B000C6005F1008001F30BD05C030DE05883064
:1003C000C505C1000030C300C70008002F30BD05BF
:1003D000C030DE051030C505C1000030C300C700C5
:1003E00008004F30BD05C030DE053030C505C10006
:1003F0000030C300C70008008F30BD05C030DE05E7
:10040000C030C505C1000030C300C700080010306F
:1004100085060230870608002030850600308706F2
:100420000800213085060030870608000230850666
:10043000023087060800003085060C308706080069
:10044000003085060130870608000030850621301F
:1004500087060800003085061830870608003D181A
:10046000AB21BD18B7213D19C321BD19CF213D1ABC
:10047000DB21BD1AE6213D1BF121BD1BFC2108003B
:10048000B601B301B4013C1C482ABC01BC144A2A81
:10049000BC013C143C08B60064004E2A4F2A502A86
:1004A000512A522AFF30B41B8500B41F8501B30BBB
:1004B0004C2AB40B4C2A0310B60CB608031D4C2A68
:1004C0000030BB003C08BA007B21080005125C1814
:1004D0000516DC1C8512DC1885165C1D05105C19E0
:1004E0000514DC1D8510DC1985145C1E87105C1A50
:1004F0008714DC1E0711DC1A07155C1F07105C1B34
:100500000714DC1F8712DC1B871608008F080319ED
:1005100008008F0178308E00C80FB02CC80A441C28
:10052000B62A461CA72ACA1C982ACA014A15C42AF8
:100530004A1D9D2ACA01CA15C42ACA1DA22ACA0177
:100540004A16C42A4A1EC42ACA01CA14C42A4A1D09
:10055000AC2ACA014A16C42ACA1DB12ACA014A16BF
:10056000C42A4A1EC42ACA01CA14C42ACA1CBB2AE5
:10057000CA014A15C42A4A1DC02ACA01CA15C42A7A
:100580004A1EC42ACA014A15C41CEB2AC61CDC2A0E
:10059000CB1CCD2ACB014B15F92A4B1DD22ACB01FE
:1005A000CB15F92ACB1DD72ACB014B16F92A4B1EA6
:1005B000F92ACB01CB14F92A4B1DE12ACB014B16AA
:1005C000F92ACB1DE62ACB014B16F92A4B1EF92A34
:1005D000CB01CB14F92ACB1CF02ACB014B15F92AFD
:1005E0004B1DF52ACB01CB15F92A4B1EF92ACB015D
:1005F0004B15441D202B461D112BCC1C022BCC016E
:100600004C152E2B4C1D072BCC01CC152E2BCC1DA5
:100610000C2BCC014C162E2B4C1E2E2BCC01CC14AB
:100620002E2B4C1D162BCC014C162E2BCC1D1B2B10
:10063000CC014C162E2B4C1E2E2BCC01CC142E2B69
:10064000CC1C252BCC014C152E2B4C1D2A2BCC0160
:10065000CC152E2B4C1E2E2BCC014C15C41D562B0D
:10066000C61D472BCD1C382BCD014D155F13642BB8
:100670004D1D3D2BCD01CD15642BCD1D422BCD0144
:100680004D16642B4D1E642BCD01CD14642B4D1DD6
:100690004C2BCD014D16642BCD1D512BCD014D168C
:1006A000642B4D1E642BCD01CD14642BCD1C5B2B14
:1006B000CD014D15642B4D1D602BCD01CD15642B47
:1006C0004D1E642BCD014D155F1B8D2B441E8D2BB4
:1006D000461E7E2BCE1C6F2BCE014E159B2B4E1D26
:1006E000742BCE01CE159B2BCE1D792BCE014E1631
:1006F0009B2B4E1E9B2BCE01CE149B2B4E1D832B72
:10070000CE014E169B2BCE1D882BCE014E169B2B59
:100710004E1E9B2BCE01CE149B2BCE1C922BCE01BA
:100720004E159B2B4E1D972BCE01CE159B2B4E1E8F
:100730009B2BCE014E15C51DC22BC71DB32BCF1C45
:10074000A42BCF014F15D02B4F1DA92BCF01CF15B7
:10075000D02BCF1DAE2BCF014F16D02B4F1ED02B41
:10076000CF01CF14D02B4F1DB82BCF014F16D02B5C
:10077000CF1DBD2BCF014F16D02B4F1ED02BCF013D
:10078000CF14D02BCF1CC72BCF014F15D02B4F1D13
:10079000CC2BCF01CF15D02B4F1ED02BCF014F1517
:1007A000451EF72B471EE82BD01CD92BD001501526
:1007B000052C501DDE2BD001D015052CD01DE32BB0
:1007C000D0015016052C501E052CD001D014052C3C
:1007D000501DED2BD0015016052CD01DF22BD00151
:1007E0005016052C501E052CD001D014052CD01C01
:1007F000FC2BD0015015052C501D012CD001D0151B
:10080000052C501E052CD0015015C51E2C2CC71EC2
:100810001D2CD11C0E2CD10151153A2C511D132C1D
:10082000D101D1153A2CD11D182CD10151163A2CD9
:10083000511E3A2CD101D1143A2C511D222CD10138
:1008400051163A2CD11D272CD10151163A2C511E8C
:100850003A2CD101D1143A2CD11C312CD101511593
:100860003A2C511D362CD101D1153A2C511E3A2C5F
:10087000D1015115451F622C471F532CD21C442C0B
:10088000D2015215DF13702C521D492CD201D21502
:10089000702CD21D4E2CD2015216702C521E702C70
:1008A000D201D214702C521D582CD2015216702C29
:1008B000D21D5D2CD2015216702C521E702CD2010A
:1008C000D214702CD21C672CD2015215702C521DE0
:1008D0006C2CD201D215702C521E702CD2015215E4
:1008E000DF1B992CC51F992CC71F8A2CD31C7B2C6E
:1008F000D3015315A72C531D802CD301D315A72C3E
:10090000D31D852CD3015316A72C531EA72CD3011E
:10091000D314A72C531D8F2CD3015316A72CD31DF2
:10092000942CD3015316A72C531EA72CD301D314F8
:10093000A72CD31C9E2CD3015315A72C531DA32CDD
:10094000D301D315A72C531EA72CD3015315722105
:100950004008C4004108C5005F18DF145F1CDF10A9
:100960004808C9000C304A05031D05120C304B0520
:10097000031D85120C304C05031D05100C304D0570
:10098000031D85100C304E05031D87100C304F05DC
:10099000031D07110C305005031D07100C305105C5
:1009A000031D87120C305205031D07120C3053052E
:1009B000031D871149080E0203180A2D12304A053B
:1009C000031D051612304B05031D851612304C050C
:1009D000031D051412304D05031D851412304E05FC
:1009E000031D871412304F05031D071512305005E3
:1009F000031D071412305105031D871612305205CE
:100A0000031D071612305305031D8715FF304802DA
:100A1000031908008F08031D0800812049080E02F1
:100A2000031C0A2D18304A05031D051206304A051D
:100A3000031D051618304B05031D851206304B05A6
:100A4000031D851618304C05031D051006304C0596
:100A5000031D051418304D05031D851006304D0586
:100A6000031D851418304E05031D871006304E05F2
:100A7000031D871418304F05031D071106304F055D
:100A8000031D071518305005031D071006305005CB
:100A9000031D071418305105031D87120630510538
:100AA000031D871618305205031D07120630520524
:100AB000031D071618305305031D87110630530513
:060AC000031D871508006C
:084000000400030006000000AB
:02400E00CC33B1
:10420000010078007A007C007E007B0079007F004E
:104210007D007A0078007E007C007D007F007900C0
:104220000200F200F600FA00FE00F200F600FA00CA
:10423000FE00F200F600FA00FE00F200F600FA00BE
:10424000FF00050005000500050009000900090040
:1042500009000D000D000D000D00110011001100EE
:104260000100FF00FF00FF00FF00FF00FF00FF0054
:10427000FF00FF00FF00FF00FF00FF00FF00FF0046
:10428000FF007B00FF00FF00FF00FF00FF00FF00BA
:10429000FF00FF00FF00FF00FF00FF00FF00FF0026
:1042A000FF00FE00FF00FF00FF00FF00FF00FF0017
:1042B000FF00FF00FF00FF00FF00FF00FF00FF0006
:1042C000FF001100FF00FF00FF00FF00FF00FF00E4
:1042D000FF00FF00FF00FF00FF00FF00FF00FF00E6
:1042E000FF00FF00FF00FF00FF00FF00FF00FF00D6
:1042F000FF00FF00FF00FF00FF00FF00FF00DD00E8
:00000001FF
